:100000000C9434050C9495050C947F080C9495057C
:100010000C9495050C9495050C9495050C949505F8
:100020000C9495050C9495050C9495050C94CB15A2
:100030000C9495050C9467230C9495050C949505E8
:100040000C9495050C9495050C9495050C94BC2383
:100050000C9495050C9495050C9495050C949505B8
:100060000C9495050C9495050C9495050C949505A8
:100070000C949505510A530A5F0A5F0A5F0A5F0AEA
:100080005F0A5F0A550A570A590A5F0A5F0A530A4C
:10009000610A5F0A5F0A1B0A510A5F0A5F0A570A70
:1000A0005F0A5F0A5F0A5F0A5F0A5F0A590A510A1C
:1000B0003D0A5F0A410A5F0A5F0A5F0A1D0A550A84
:1000C0005F0A5F0A4B0A5F0A5F0A5F0A1F0A5D0A3E
:1000D0005F0A3F0A5F0A530A5F0A5F0A4F0A430A30
:1000E0005F0A450A570A5F0A5F0A5F0A4D0A470A14
:1000F0005F0A5F0A5F0A5F0A5F0A5F0A5F0A490ACE
:100100005F0A210A5F0A5F0A550A5F0A5F0A5D0AF1
:100110005F0A5F0A5F0A5F0A5F0A5F0A5F0A5F0A97
:100120005F0A230A5F0A5F0A5F0A4B0A5F0A5F0AD7
:100130005F0A5F0A5F0A5F0A5F0A5F0A5F0A5F0A77
:10014000250A5F0A270A290A5F0A5F0A5F0A2B0A43
:100150002D0A2F0A5F0A310A330A5F0A5F0A5F0A13
:100160005B0A350A5F0A390A370A3B0A5F0A5F0AE7
:100170005F0A5F0A5D0A850A930A9F0A9F0A770A47
:100180009F0A9F0A9F0A9F0A9F0A9F0A9F0A9F0A27
:100190009F0A9F0A9F0A9F0A9F0A790A9F0A7B0A61
:1001A0009F0A9F0A9F0A9F0A970A9F0AAE0A950A0A
:1001B0009F0A9F0A9F0A9F0A9F0A9F0A9F0A9F0AF7
:1001C0009F0A9F0A9F0A9F0A9F0A6F0A8B0A7D0A4D
:1001D0008F0A9F0A7F0A9F0A830A9F0A8D0A810A53
:1001E000910A870A890A9F0A9F0A9F0A9F0A9F0A03
:1001F0009F0A9F0A710A730A750A990A9B0A9F0A45
:100200009F0A9F0A9D0A7D0B9B0BA70BCB0BDB0B59
:10021000E70B030C1A0C3D0C5A0CE50C110D8B0D61
:10022000BD0DA70DCE0DE00DE80DEE0DF20DF80D94
:10023000540E560E580E5A0E9A0E620E620E620E32
:100240005C0E5E0E600E3114581450155814501583
:10025000A414C71450151E152D156E196E19981972
:100260009819F3191E1C1E1C1E1C271A1E1C121B7B
:10027000121BD81B1E1CED1B0B1C007B460102032E
:10028000763A687F6577482B353B6978796439140D
:100290001E3C6A7A1D16041A1F3D6B061B070821B7
:1002A000203E6C2C19091715223F6D11050B0A1CF5
:1002B00023406E7E100D182425416F360E0C122738
:1002C00026427037380F33132D43717534322F2E79
:1002D00044727C7D28303174457351504A524D49E7
:1002E0002A5466594F5C5F4C4B4E62635A5D5E60A8
:1002F000295367585B56576147554842403E3C3A40
:100300003B456843413F3D2B357E697A790078143F
:100310001E7C6A7B1D16041A1F7F6B061B070821B3
:10032000204D6C2C19091715224A6D11050B0A1C5A
:10033000234C6E49100D182425516F360E0C1227D0
:10034000264F7037380F33132D52717534502F2EBE
:100350004E72397D283065314B735464586776018D
:100360002A773259745C5F66020362635A5D5E608D
:10037000295344575B565561474680291E1F20214B
:100380002223242526272D2E2A2B141A0815171C64
:10039000180C12132F302878041607090A0B0D0EBB
:1003A0000F33343579311D1B0619051110363738D6
:1003B0007D557A2C393A3B3C3D3E3F4041424353C8
:1003C000475F6061565C5D5E57595A5B62634648A1
:1003D000324445677B7F650301025250514F686983
:1003E0006A6B6C6D6E6F7071725800494C754A4D36
:1003F000734B4E767C777E7466547225303258206B
:1004000000623A25303458200065253032582000EB
:100410002146554C4C2120002146462120007725BD
:100420003032582000214353335F4630210A0021E7
:100430004353335F5245414459210A00214353320B
:100440005F45305F4630210A00214353325F46301A
:10045000210A00214353325F4530210A00214353D2
:10046000325F494E4954210A00214353315F4530E0
:100470005F25303258210A000A5B4F56525D20003A
:100480004C2575200053257520000A49443A253033
:1004900034582825642920004D6F7573653A206E05
:1004A0006F7420737570706F727465640A005225E2
:1004B0007520005725752000572575200057257594
:1004C00020005825752000412575200049257520FC
:1004D000005B4348475D20000A5052543A253032B1
:1004E00058204953523A2530345820005B52535417
:1004F0005D20000A4552523A253032582049535265
:100500003A2530345820000A4B6579626F61726475
:100510002073746172742E0A000A55534220636F6F
:100520006E666967757265642E0A000A0A544D4B3F
:100530003A30616230656266382F4C5546410A0A8E
:10054000003403490042004D0020005000430020C9
:10055000006B006500790062006F0061007200644A
:1005600000200063006F006E00760065007200746A
:10057000006500720000000E0374002E006D002E56
:10058000006B002E0000000403090409027400043B
:100590000100A0320904000001030101000921113A
:1005A0000100012240000705810308000A09040137
:1005B000000103000000092111010001223600079B
:1005C00005820308000A0904020002030000000972
:1005D00021110100012222000705830320000107E9
:1005E00005030320000109040300010300000009C2
:1005F00021110100012239000705840320000112A6
:1006000001100100000008EDFEEE1B0100010200D8
:100610000105010906A101050719E029E7150025D3
:1006200001950875018102050819012905950575CF
:100630000191029501750391010507190029F7152C
:1006400000250195F875018102C00631FF0974A1EA
:10065000010975150026FF009520750881020976AD
:10066000150026FF00952075089102C0050109803C
:10067000A10185021601002637001A81002AB70061
:10068000751095018100C0050C0901A101850316B3
:100690000100269C021A01002A9C02751095018116
:1006A00000C005010906A101050719E029E71500A9
:1006B00025019508750181029501750881010508DC
:1006C000190129059505750191029501750391019F
:1006D0000507190029FF150026FF009506750881FA
:1006E00000C0636F6E73756D65723A2025303458A3
:1006F0000A0073797374656D3A20253034580A0006
:100700000A002530325820006B6579626F6172648F
:100710003A20004C45443A20253032580A00253012
:1007200032583A202530386225730A00722F632030
:1007300030313233343536370A0064656C5F6B65AF
:10074000795F6269743A2063616E27742064656C16
:100750003A20253032580A006164645F6B65795F26
:100760006269743A2063616E2774206164643A2080
:10077000253032580A003F00433E20004C25640AD1
:10078000000A092D20436F6E736F6C65202D0A459A
:1007900053432F713A09717569740A000A092D20B3
:1007A0004D61676963202D0A643A09646562756763
:1007B0000A783A096465627567206D6174726978B8
:1007C0000A6B3A096465627567206B6579626F61CF
:1007D00072640A6D3A096465627567206D6F75739E
:1007E000650A763A0976657273696F6E0A733A091B
:1007F0007374617475730A633A09636F6E736F6C17
:1008000065206D6F64650A302D343A096C61796535
:1008100072302D34284631302D4634290A50617506
:10082000733A09626F6F746C6F616465720A6E3A35
:10083000094E4B524F0A003F004E4B524F3A206F29
:1008400066660A004E4B524F3A206F6E0A0074697A
:100850006D65725F72656164333228293A202530F4
:10086000346C580A006B6579626F6172645F6E6BFD
:10087000726F3A2025580A006B6579626F61726465
:100880005F69646C653A2025580A006B6579626F70
:100890006172645F70726F746F636F6C3A20255879
:1008A0000A00686F73745F6B6579626F6172645F71
:1008B0006C65647328293A2025580A000A092D20FE
:1008C000537461747573202D0A004743433A2035F1
:1008D0002E342E30204156522D4C4942433A20327C
:1008E0002E302E30204156525F415243483A20610B
:1008F000767233350A004F5054494F4E533A204CCC
:100900005546412045585452414B455920434F4E7E
:10091000534F4C4520434F4D4D414E44204E4B527A
:100920004F204B45594D41505F53454354494F4E1D
:1009300020424F4F544C4F414445525F53495A4512
:100940000A004255494C443A203061623065626683
:1009500038202831313A35373A3230204D6179200C
:1009600032322032303230290A005649443A20309F
:10097000784645454428742E6D2E6B2E292050490B
:10098000443A203078316265652849424D20504311
:10099000206B6579626F61726420636F6E76657239
:1009A00074657229205645523A2030783030303103
:1009B0000A00444553433A20636F6E766572742093
:1009C00049424D205043206B6579626F617264200B
:1009D000746F205553420A000A092D205665727320
:1009E000696F6E202D0A000A6D6F7573653A206F6E
:1009F00066660A000A6D6F7573653A206F6E0A00AD
:100A00000A6B6579626F6172643A206F66660A00EC
:100A10000A6B6579626F6172643A206F6E0A000A30
:100A20006D61747269783A206F66660A000A6D61BA
:100A3000747269783A206F6E0A000A64656275679D
:100A40003A206F6E0A000A64656275673A206F6625
:100A5000660A000A0A626F6F746C6F616465722EB9
:100A60002E2E2000433E200011241FBECFEFD4E0E5
:100A7000DEBFCDBF04B603FE41C0809188039091D4
:100A80008903A0918A03B0918B038730904BA740D4
:100A9000B04BA1F5109288031092890310928A033B
:100AA00010928B0314BE0FB6F894A8958091600045
:100AB000886180936000109260000FBE1092010860
:100AC00010920008E3E0F0E089E080935700E491A1
:100AD000E695E370E150E33040F4F0E0EE0FFF1FE5
:100AE000E35DFE4F8081918102C080E090E1E0E013
:100AF000F0E8E81BF90BF695E795099511E0A0E001
:100B0000B1E0E4EAFBE402C005900D92A433B10722
:100B1000D9F723E0A4E3B1E001C01D92A838B207E1
:100B2000E1F70E9450110C94D0250C940000FF9323
:100B3000EF93E0913401F0913501309709F0099578
:100B4000EF91FF910895FC018591803011F0EFDF66
:100B5000FBCF0895FF27E0E230E247FF0CC041954C
:100B600097FF09C0EDE26095709580959095611DA5
:100B7000711D811D911D27FF02C0219530E350E2B8
:100B8000AA27660F771F881F991FAA1FA41710F0A6
:100B9000A41B63955A95A9F7AA3008F0A95FA05D38
:100BA000AF93F395611571058105910541F7ED321C
:100BB00011F4EF93F395F21718F43F93F395FBCFED
:100BC0008F91B5DFFA95E1F70895E991F991859153
:100BD000803021F0853219F0AADFF9CF089520E0A6
:100BE000E89455915532C1F3503311F468945591FE
:100BF0005A3348F4505390F3220F022E220F220F43
:100C0000200D250FF4CF0EF421958991999153363B
:100C100019F3533729F1533559F1BC018827992726
:100C2000E8945C3621F489919991689455915436F1
:100C300039F446EF7EF077FF0DC08FEF9FEF0AC0CB
:100C400055374AE039F0583540E121F0523642E05C
:100C500009F00895FF93EF937DDFEF91FF91B7CFF8
:100C6000FF93EF93FC0181918030B9F360DFFBCFFC
:100C7000FF93EF9368DFF1CFDF93CF93CDB7DEB76C
:100C80002596A3DFCF91DF91089590914101923095
:100C900081F09330D1F0913031F5E72FF0E0B3E0FF
:100CA000EE0FFF1FBA95E1F7E60FF11DE658FC4F76
:100CB00017C0E72FF0E0A3E0EE0FFF1FAA95E1F7C2
:100CC000E60FF11DE650FD4F0BC0E72FF0E073E09B
:100CD000EE0FFF1F7A95E1F7E60FF11DE658FD4F85
:100CE000E491E03819F480E090E0089590E023E08A
:100CF000880F991F2A95E1F72E2F207730E044E0E6
:100D0000359527954A95E1F7820F931F54E0880F98
:100D1000991F5A95E1F7EF709C012E0F311DF901D3
:100D2000EE0FFF1FE050F84985919491089559986E
:100D3000519A08955198599A08955898509A08953B
:100D40005098589A08955198599A85E08A95F1F7E4
:100D5000000089B18695817008955098589A85E071
:100D60008A95F1F7000089B181700895CF93DF93E0
:100D7000EC010E94A306882341F0209731F085E022
:100D80008A95F1F700002197F4CFCE01DF91CF9142
:100D90000895CF93DF93C2E3D0E00E94A3068111B0
:100DA00008C0209731F085E08A95F1F7000021977F
:100DB000F4CFCE01DF91CF9108952E9826982F98E9
:100DC00027980E9497060E94A006E9E6F0E080813D
:100DD00088608083E9980895E19AE99A0E949A06CA
:100DE0000C94A006E9980E9497060C94A006CF9355
:100DF000DF932FB7F894C0910201D0910301CE0187
:100E0000882781159F4F19F080E09FEF02C08FEF78
:100E100090E08C2B9D2B90930301809302012FBFB8
:100E2000CE0199278F3F910581F5CD2FDD27C03F5A
:100E3000D10551F0CF3FD10509F451C08091750320
:100E4000C034D10599F407C08091750380FF33C089
:100E500088E194E004C080FF2EC080E194E09F937D
:100E60008F930E943C060F900F9025C080FF37C0E3
:100E7000DF93CF9389E094E09F938F930E943C0689
:100E80000F900F900F900F902AC0CE018F6F019698
:100E900099F08091750380FF0CC0DF93CF9381E0C0
:100EA00094E09F938F930E943C060F900F900F90B9
:100EB0000F90CD2F01C0CFEF8091750380FF0CC044
:100EC0001F92CF938AEF93E09F938F930E943C06EB
:100ED0000F900F900F900F908C2F90E002C08FEF2B
:100EE0009FEFDF91CF910895CF93CAE1C15069F090
:100EF0000E94F7068F3F2FEF920749F48FE99FE09A
:100F00000197F1F700C00000F1CF8FEF9FEFCF9175
:100F1000089510923A0110923901109238011092FE
:100F2000370180E090E890930101809300018FEFFA
:100F30009FEF90930301809302010895EF92FF9237
:100F40000F931F93CF93DF93082F10923701809157
:100F5000750380FF0CC01F920F938EE194E09F9366
:100F60008F930E943C060F900F900F900F90E9987E
:100F70000E9497060E94A0068FE891E00197F1F782
:100F800000C000000E949D068FE891E00197F1F7F4
:100F900000C000000E949A0680E197E20E94B60617
:100FA000892B11F481E07FC0C0E0D0E0FF24F394EE
:100FB00010E0EE24E39490E59A95F1F7C8010C2E29
:100FC00002C0959587950A94E2F780FF04C0FE243D
:100FD0000E94A00602C00E949D060E94C906892B9D
:100FE00011F482E060C082E390E00E94B606892B93
:100FF00011F483E058C02196C830D105E1F680E5B0
:101000008A95F1F7FF2019F00E94A00602C00E9405
:101010009D060E94C906892B11F484E044C082E336
:1010200090E00E94B606892B11F485E03CC090E563
:101030009A95F1F70E94A0060E94C906892B11F427
:1010400086E031C082E390E00E94B606892B19F059
:10105000C2E3D0E009C087E026C0209759F025E020
:101060002A95F1F7000021970E94AD068111F5CF76
:10107000CD2B11F488E017C00E94C906892B19F006
:10108000C2E3D0E009C089E00EC0209759F085E0A6
:101090008A95F1F7000021970E94AD068823A9F3F5
:1010A000CD2BB9F48AE080933701809137018061BC
:1010B000809337010E949A060E94A006E19AE99A5D
:1010C0008FEF9FEFDF91CF911F910F91FF90EF90E6
:1010D00008958FEF9FEF90930301809302010E9488
:1010E00089070E949A060E94A006E19AE99ADF9178
:1010F000CF911F910F91FF90EF900C9474071F9266
:101100000F920FB60F9211242F933F934F935F933B
:101110008F939F9329B19091760340910001509154
:1011200001014115504819F49093360111C0809186
:101130003601981769F08F5F981751F08091000180
:101140009091010190933A018093390180E2DDC0D2
:1011500080910001909101019695879590930101EE
:101160008093000120FF09C080910001909101014E
:10117000906890930101809300018091000190910B
:10118000010199278038910509F4F9C0A8F480324B
:10119000910509F4F4C038F4009709F4F0C04097C1
:1011A00009F489C0A9C08034910509F4E8C08035EC
:1011B000910509F480C0A0C0803C910539F150F43C
:1011C0008039910509F477C0803A910509F094C0FF
:1011D00084E64DC0803D910509F46DC0803E9105C7
:1011E00009F08AC0809100019091010190933A0129
:1011F000809339018091000190910101892F9927F5
:10120000909301018093000183E252C084E64999E2
:101210000FC0882369F095E09A95F1F7000081509E
:10122000F6CF882349F095E09A95F1F700008150B8
:101230004999F7CF8111A3C08091000190910101DC
:1012400090933A01809339018091000190910101BE
:10125000892F9927909301018093000182E228C091
:10126000882379F095E09A95F1F700008150499B29
:10127000F7CF07C0882349F095E09A95F1F7000071
:1012800081504999F7CF81117AC0809100019091E6
:10129000010190933A01809339018091000190916E
:1012A0000101892F9927909301018093000181E228
:1012B0008093380133C08091000190910101909397
:1012C0003A0180933901809100019091010197FFCB
:1012D00002C080E101C081E180933801809100016A
:1012E0009091010146E0969587954A95E1F7909394
:1012F00001018093000112C08091000190910101D1
:1013000090933A018093390180E88093370180916E
:10131000370190E0982F88278F6F27C080910001B8
:101320009091010199278F3F910511F480EFEDCF46
:10133000809103018F3F31F0809102018F3F11F0C6
:1013400080E4E3CF8091020190910301982F8827D8
:1013500090930301809302012091000130910101DB
:101360008091020190910301822B9093030180935D
:10137000020180E090E890930101809300019F9129
:101380008F915F914F913F912F910F900FBE0F90D2
:101390001F901895CF93C82F8DEE0E949E078A3F0D
:1013A000910521F48C2FCF910C949E07CF91089535
:1013B000E82FE695E695E695EF70F0E0EB5BFE4FE3
:1013C0004081282F277081E090E002C0880F991F8C
:1013D0002A95E2F7242F30E028233923232B11F418
:1013E000842B80830895E82FE695E695E695EF70C7
:1013F000F0E0EB5BFE4F2081382F377081E090E00A
:1014000002C0880F991F3A95E2F7422F50E0482317
:101410005923452B19F08095822380830895482F06
:1014200050E0FA013397E138F10508F048C0E65C76
:10143000FF4F0C94CA2587E108958FE108958CE54C
:10144000089580E6089582E6089587E2089583E589
:1014500008958FE2089589E3089587E308958FE35F
:10146000089587E408958FE4089586E508958EE54C
:1014700008958FE7089580E0089585E608958EE643
:1014800008958FE6089580E3089588E3089580E441
:10149000089588E4089580E5089587E508958FE527
:1014A000089588E1089588E0089580E2089580E134
:1014B000089589E108958DE6089588E208958F776B
:1014C00008958FE00895CF93482F50E0FA017C975C
:1014D000E834F105A0F5E554FF4F0C94CA2585E5E5
:1014E0003EC08AE53CC08BE53AC08CE538C08DE54E
:1014F00036C08EE534C08FE532C080E630C081E66C
:101500002EC082E62CC083E62AC08FE628C081E781
:1015100026C082E724C084E722C085E720C087E791
:101520001EC088E71CC08AE71AC08CE718C08FE786
:1015300016C080E714C089E712C08BE710C0C82F1F
:101540001F928F9389E694E09F938F930E943C06AD
:101550000F900F900F900F908C2F01C084E5CF91CA
:1015600008950F931F93CF93DF930E9495238C01CF
:101570000E94F706EC01019631F4C8010E94AD23E8
:10158000843F9140A8F3CE01DF91CF911F910F913D
:1015900008950E94DD060C94EC068091750381602D
:1015A00080937503E5E4F1E0119281E0E535F807F9
:1015B000D9F70895E82FF0E0EB5BFE4F80810895A6
:1015C000E5E4F1E0119281E0E535F807D9F70895F7
:1015D000982F80914101823048F092FB882780F952
:1015E00090FD826091FD84600C94CA090895CF93A8
:1015F000DF9380913701882371F1809139019091B7
:101600003A01209137019F938F931F922F9383EF7D
:1016100094E09F938F930E943C06809137018075E0
:101620000F900F900F900F900F900F9071F480918A
:1016300040018B3051F48CEE94E09F938F930E9485
:101640003C06109240010F900F90109237011092BB
:101650003A011092390180913801882309F440C081
:1016600090913801809144019817D1F1809139010E
:1016700090913A01209138019F938F931F922F935D
:1016800088ED94E09F938F930E943C0680914401E3
:101690000F900F900F900F900F900F9085FF04C048
:1016A0009091380194FD06C084FF12C080913801EA
:1016B00085FF0EC0809140018B3051F481ED94E0A4
:1016C0009F938F930E943C06109240010F900F90C1
:1016D000809138018093440110923A0110923901AF
:1016E000E09140018E2F90E08C30910508F026C3E8
:1016F000FC01ED5FFE4F0C94CA250E94F2060E9489
:1017000095239F938F938CEC94E09F938F930E94EB
:101710003C061092410110924301109242010E9436
:10172000E00A0E941E190E94952390933F01809326
:101730003E0181E065C080913E0190913F010E9491
:10174000AD23893E934008F4F9C282E031C00E9483
:1017500089070E94EC068FE99FE00197F1F700C02E
:1017600000008FEF0E949E078A3F910511F486E0EA
:1017700001C083E0809340010E9495239F938F9343
:1017800087EC94E09F938F930E943C060F900F90FC
:101790000F900F90D3C20E94F2062E98269A2F988F
:1017A000279A0E94952390933F0180933E0184E005
:1017B00080934001C3C280913E0190913F010E94FD
:1017C000AD23853F914008F4B9C285E0F1CF2E9852
:1017D00026982F9827980E9489070E94EC060E945D
:1017E00095239F938F9382EC94E09F938F930E9415
:1017F0003C060E94952390933F0180933E0186E032
:1018000080934001C3CF0E94F706019609F496C267
:101810000E9495239F938F938DEB94E09F938F93DA
:101820000E943C060E94952390933F0180933E01C5
:1018300087E0E6CF80913E0190913F010E94AD2369
:10184000853F914018F089E0809340010E94F7069F
:10185000019609F473C20E9495239F938F9388EB9E
:1018600094E09F938F930E943C060E94952390934F
:101870003F0180933E0188E0C3CF80913E0190916B
:101880003F010E94AD23853F914018F089E080938D
:1018900040010E94F706019609F450C20E94952368
:1018A0009F938F9383EB94E09F938F930E943C06CA
:1018B00089E0A6CF82EF0E949E078F3F2FEF92070D
:1018C00089F08A3F910589F40E94B10A8F3F3FEF6A
:1018D000930771F0D82FCC270E94B10A9E01282BC4
:1018E000C90108C08FEF9FEF05C08EEF9FEF02C0C8
:1018F00080E090E090934301809342010E94952301
:101900009F938F938EEA94E09F938F930E943C065F
:1019100080914201909143010F900F900F900F9092
:10192000009711F482E02BC08F3F3FEF930711F433
:1019300081E025C08E3F2FEF9207A1F38F3F9105E5
:1019400059F488E994E09F938F930E943C0610928B
:1019500041010F900F901FC09C0125583B4A223037
:10196000310580F480EF0E949E078A3F9105D1F6F1
:1019700083E00E949E078A3F9105A1F683E0809351
:10198000410109C0803B3FEB9307C1F388278115D4
:101990009F4BA1F3C7CF809141011F928F938091FC
:1019A00043018F93809142018F938AE894E09F9343
:1019B0008F930E943C068AE0809340010F900F9025
:1019C0000F900F900F900F90B9C10E9495239F9395
:1019D0008F9385E894E09F938F930E943C060F902D
:1019E0000F900F900F9080914101823029F0833049
:1019F00039F488EF0E949E070E9496160E94E80A1A
:101A00008BE0809340010E9495239F938F9380E801
:101A100094E09F938F930E943C060F900F900F903D
:101A20000F900E94F7069C012F3F9FEF390709F4A2
:101A300085C12115310519F02F3F310569F40E9448
:101A4000E00A0E941E1988E794E09F938F930E94FA
:101A50003C060F900F9072C190914101923009F4B1
:101A60004DC0933009F4CCC0913009F067C190911A
:101A70003D01923099F028F4992341F09130C1F062
:101A80003AC0933081F1943091F135C0803E21F01D
:101A9000813E51F482E005C081E003C08D31F9F44C
:101AA00083E080933D014AC187FFE4C08F770EC178
:101AB000863309F118F48A3229F41DC08A3AD9F024
:101AC000863BC9F087FD05C00E94630A0E94D809C1
:101AD00012C08F770E94630A0E94F3090CC08D39EF
:101AE00051F484E0DECF853431F485E5C3C085341C
:101AF00011F485E5EBC010923D0120C1E0913C015D
:101B00004E2F50E04930510508F077C0FA01E15FEF
:101B1000FE4F0C94CA25803E69F030F4833871F092
:101B2000843871F48FE757C0813E31F0803F41F433
:101B300081E05BC082E059C084E057C082E04BC0C6
:101B400087FF98C00E94E00A8DE594E098C089352F
:101B500009F453C0803F19F0823119F44EC083E07C
:101B600044C010923C0187FD03C00E940F0A82C04E
:101B70000E94E00A83E594E082C0833821F0843833
:101B800021F48FE738C082E036C010923C0187FF15
:101B90009DC00E94E00A89E494E071C010923C016B
:101BA000823109F4CBC0893509F4C8C087FD03C070
:101BB0000E940F0A8BC00E94E00A8CE394E05FC091
:101BC000843121F0803FC9F486E00FC085E00DC06C
:101BD000873799F480E00E94D8090FC0843169F4F6
:101BE00087E003C0803F49F488E080933C01A6C0B1
:101BF000873719F480E00E94F30910923C019EC0DF
:101C000090913B01913009F443C038F0923009F4CF
:101C100063C0933009F47FC091C0863809F168F43D
:101C20008338D1F020F4803819F582E06CC0843814
:101C3000A9F08538E9F48BE01DC08C38A9F030F4A8
:101C4000873881F08B38A1F481E014C08D3871F0B1
:101C5000803F71F481E057C082E00CC08FE70AC07A
:101C600086E008C080E006C089E004C08AE002C0C7
:101C700087FD03C00E94D80961C08FE294E09F9362
:101C80008F930E943C060F900F901092400156C017
:101C9000482F50E0FA01E358F109EB30F10590F4D8
:101CA000E85EFE4F0C94CA2582E045C08FE743C032
:101CB0008BE041C086E03FC081E03DC089E03BC091
:101CC0008AE039C010923B0187FD03C00E94F309EE
:101CD00035C085E294E0D3CF853279F030F4863197
:101CE00071F08E3199F480E00BC0863221F0803F94
:101CF00069F483E008C08DE503C083E501C081E598
:101D00000E94D80905C080933B0118C00E94E00AD8
:101D100010923B0113C08E3169F020F48631B1F787
:101D200081E509C0853221F0863281F78DE503C057
:101D300083E501C080E00E94F309EACF81E0DF91F2
:101D4000CF9108958091790208950895CF93DF93FC
:101D500000D01F92CDB7DEB720917F03243021F54C
:101D600023E029839B838A8382E08093E9008FEFBD
:101D70009091E800815095FD06C095ED9A95F1F798
:101D800000008111F5CF8091E80085FF0DC040E093
:101D900050E063E070E0CE0101960E940213809152
:101DA000E8008E778093E8000F900F900F90DF91FE
:101DB000CF910895CF93DF9300D01F92CDB7DEB7B8
:101DC00020917F03243029F522E02983805891094E
:101DD0009B838A832093E9008FEF9091E8008150E4
:101DE00095FD06C095ED9A95F1F700008111F5CFAC
:101DF0008091E80085FF0DC040E050E063E070E0B6
:101E0000CE0101960E9402138091E8008E778093A4
:101E1000E8000F900F900F90DF91CF910895CF932E
:101E2000DF93EC0190917F03943009F048C08091DA
:101E300014018823D9F0809115018823B9F090937B
:101E4000E90081E8815049F09091E80095FD05C0D6
:101E50009AE29A95F1F700C0F5CF8091E80085FFEE
:101E60002EC040E050E060E270E019C081E0809355
:101E7000E90081E8815059F09091E80095FD07C094
:101E8000EFE3F1E03197F1F700C00000F3CF80916C
:101E9000E80085FF14C040E050E068E070E0CE014B
:101EA0000E9402138091E8008E778093E80080E220
:101EB000FE01A9E5B2E001900D928A95E1F7DF916C
:101EC000CF910895CF93C0915701C1110BC00E94CB
:101ED000A123643C79408105910520F081E0809345
:101EE0005701C1E08C2FCF910895FF920F931F935C
:101EF000CF93DF93D82F0FB607FE83C080917F0367
:101F0000843081F08091070190E0019620910901D1
:101F100030E0822393232091080130E08217930759
:101F200009F0C9C00E94620F811110C080910701A1
:101F300090E001962091090130E0822393232091C3
:101F4000080130E08217930709F0B5C00E9495237D
:101F50008C01C091E900CF709091EC00892F8170C5
:101F600090FD80E8C82B83E08093E90085E0F82E9F
:101F70008091EB0085FD42C08091EB0080FF3EC068
:101F80008091EE0087FF3AC080910801909107018F
:101F9000981709F457C09091E80095FF8AC0E09126
:101FA0000501F0910601E80FF11D20818F5F9091EE
:101FB00009018923809308012093F1008091E800B2
:101FC00085FDE2CF8091E80080FFDECF8091E800C0
:101FD0008E778093E800F0920401D6CF80910701BC
:101FE00090E001962091090130E082239323209113
:101FF000080130E08217930709F448C0CF70C093FE
:10200000E90040910701842F90E001962091090199
:1020100030E0822393232091080130E08217930758
:1020200009F44CC0E0910501F0910601E40FF11DA7
:10203000D083809107018F5F90910901892380935C
:1020400007013CC08091E80085FF33C0D093F100C8
:1020500081E09091F200992391F09091E80090FF37
:102060000EC09091E80095FF03C01092F100F9CFE7
:102070009091E8009E779093E800F0920401882305
:1020800009F4ACCFCF70C093E90018C0809104016F
:10209000882309F4B3CF0E9495239C0180179107F0
:1020A00011F4890165CF909104019150909304013E
:1020B000F8CF80E0CECF40910701B4CF80E0DF9130
:1020C000CF911F910F91FF900895089542E061EC28
:1020D00081E00E947B1242E061EC82E00E947B1270
:1020E00042E261EC83E00E947B1242E261EC84E018
:1020F0000C947B1280918103833009F455C030F435
:10210000813071F0823009F48EC008958A3009F46C
:102110007AC08B3009F460C0893009F09CC020C0BF
:1021200080918003813A09F096C08091E800877F12
:102130008093E8008091840390918503892B21F49A
:1021400060E289E592E003C060E080E090E070E04A
:102150000E944F138091E8008B778093E8000895E8
:1021600080918003813209F076C080918403909140
:102170008503009719F0039709F06DC08091E8007E
:10218000877F8093E8008091E80082FD05C0809100
:102190007F038111F8CF5FC08091F10080937902B5
:1021A0008091E8008B7753C080918003813A09F0D9
:1021B00052C08091840390918503892B09F04BC014
:1021C0008091E800877F8093E8008091E80080FF9D
:1021D000FCCF8091140136C0809180038132D9F503
:1021E0008091840390918503892BA9F58091E80063
:1021F000877F8093E8000E94B012809182038093D1
:1022000014010C941E1980918003813221F5809174
:10221000E800877F8093E8000E94B01280918303DA
:1022200080937A02089580918003813AA1F480918D
:10223000E800877F8093E8008091E80080FFFCCF72
:1022400080917A028093F1008091E8008E778093EC
:10225000E8000C94B012089580917902809358019F
:10226000109279020E94E00A0C941E190C942C1111
:102270000E94422380917D03882329F00E944F23EE
:1022800081110C94651208950E9463238091580176
:102290008093790208950C94441108950C944D1183
:1022A000CF9384B7877F84BF0FB6F894A8958091A9
:1022B0006000886180936000109260000FBE90E023
:1022C00080E80FB6F89480936100909361000FBE90
:1022D00085E79FE00E9415238AE091E00E94911615
:1022E0008BE295E00E94A3050E94C90A0E9445174F
:1022F0000E9468150E94BB1578940E944717809130
:102300007F03843029F00E9476160E944D11F7CF8A
:1023100089E195E00E94A3050E944E1187E095E0B7
:102320000E94A305C3E080917F03853019F40E94C9
:102330003811F9CF0E944B172091E4003091E5004D
:1023400080915501909156012817390709F464C00E
:102350008091E4009091E50090935601809355019F
:102360000E94620F882309F457C080917F03843054
:1023700009F052C08091E9008F702091EC00922FFB
:10238000917020FD90E8892BC093E9009091EB00BB
:1023900090FF3FC09091EE0097FF3BC090910801E5
:1023A00020910701291709F12091E80025FF1DC0A0
:1023B000E0910501F0910601E90FF11D30819F5F69
:1023C000209109019223909308013093F10090919C
:1023D000E80095FDE3CF9091E80090FFDFCF90916A
:1023E000E8009E779093E800D9CF9091F20099236E
:1023F00081F09091E80090FF0CC09091E80095FF6B
:1024000003C01092F100F9CF9091E8009E7790936D
:10241000E8008F708093E9000E94761684CF292F00
:10242000332723303105C9F060F42130310581F0C4
:102430002230310509F041C084E790E02BE835E017
:1024400040C021323105E1F02232310531F135C091
:1024500082E190E02FEF35E034C09927813091057B
:1024600049F028F0029749F5E1E4F5E005C0E7E816
:10247000F5E002C0E7E7F5E0849190E09F0121C01C
:1024800064307105D0F4660F771FFB01EC5DFE4FE1
:102490002081318189E090E014C06430710568F4D6
:1024A000FB01EE0FFF1FE45EFE4F20813181FB0137
:1024B000E85EFE4F808190E004C080E090E020E084
:1024C00030E0FA0131832083089584E089BD86E0FD
:1024D00089BD09B400FEFDCF8091D8008F7D809327
:1024E000D8008091E00082608093E0008091E0005D
:1024F00081FDFCCF0895982F953068F59093E90001
:10250000981739F07091EC002091ED005091F00097
:1025100003C0242F762F50E021FD02C09F5FECCF37
:102520003091EB003E7F3093EB003091ED003D7F2A
:102530003093ED003091EB0031603093EB007093FD
:10254000EC002093ED005093F0002091EE0027FD69
:10255000E5CF80E008958F708093E90081E00895D1
:102560008091800387FF11C08091E80082FD05C043
:1025700080917F038111F8CF11C08091E8008B77A3
:102580000BC080917F03882349F08091E80080FF91
:10259000F8CF8091E8008E778093E800089520912D
:1025A000E4003091E50095E64091EC00842F8170C5
:1025B00040FF23C08091E80080FD1DC080917F0313
:1025C000882399F0853099F08091EB0085FD11C04A
:1025D0004091E4005091E5002417350729F391500C
:1025E00011F09A01E1CF84E0089582E0089583E03C
:1025F000089581E0089580E008954091E80042FF49
:10260000DDCF0895CF92DF92EF92FF920F931F9349
:10261000CF93DF93EC018B017A010E94CF128111DD
:1026200035C0E114F10439F0F70180819181081B74
:10263000190BC80FD91FC12CD12C0115110529F177
:102640008091E80085FD18C08091E8008E77809326
:10265000E8000E947616E114F10449F0F701808148
:102660009181C80ED91ED182C08285E00FC00E9420
:10267000CF12882311F30AC089918093F100015091
:102680001109FFEFCF1ADF0AD8CF80E0DF91CF9199
:102690001F910F91FF90EF90DF90CF9008952091C0
:1026A0008603309187032617370748F061157105B7
:1026B00039F42091E8002E772093E80001C0B90199
:1026C000FC0120E06115710561F180917F03882391
:1026D000D9F18530D9F18091E80083FD39C080912E
:1026E000E80082FD2BC08091E80080FFEBCF809155
:1026F000F20090E06115710551F08830910538F4D1
:1027000021912093F100615071090196F3CF21E0EE
:10271000089709F020E08091E8008E778093E80028
:10272000D1CF2111D2CF0AC080917F03882361F0DD
:10273000853061F08091E80083FD0AC08091E80057
:1027400082FFF2CF80E0089582E0089583E008954B
:1027500081E008952091860330918703261737077B
:1027600048F06115710539F42091E8002E77209327
:10277000E80001C0B901FC0120E06115710579F1A3
:1027800080917F03882309F43DC0853009F43CC063
:102790008091E80083FD3AC08091E80082FD2CC062
:1027A0008091E80080FFE9CF8091F20090E0611510
:1027B000710559F08830910540F424912093F1007F
:1027C0003196615071090196F2CF21E0089709F026
:1027D00020E08091E8008E778093E800CECF211131
:1027E000CFCF0AC080917F03882361F0853061F0EC
:1027F0008091E80083FD0AC08091E80082FFF2CF5B
:1028000080E0089582E0089583E0089581E00895CE
:102810001F93CF93DF93CDB7DEB7AA970FB6F89487
:10282000DEBF0FBECDBFE0E8F3E08091F100819301
:1028300023E0E838F207C9F70E947A108091E80097
:1028400083FF2EC18091800390918103492F50E036
:102850004A30510508F024C1FA01ED5DFE4F0C9499
:10286000CA25803821F0823809F01AC108C0809149
:102870007C0390917D03992389F082600FC0809141
:1028800084038F70853008F00BC18093E90080913C
:10289000EB0085FB882780F91092E9009091E80011
:1028A000977F9093E8008093F1001092F100D1C0DF
:1028B000282F2D7F09F0F4C0882319F0823061F0B1
:1028C000EFC080918203813009F0EAC0933009F0B3
:1028D00080E080937D032EC08091820381112AC005
:1028E000809184038F702FEF280F243008F0D8C018
:1028F0008093E9002091EB0020FF1CC0933021F46D
:102900008091EB00806214C09091EB0090619093F5
:10291000EB0021E030E0A90102C0440F551F8A9569
:10292000E2F74093EA001092EA008091EB008860A1
:102930008093EB001092E9008091E800877F8093FC
:10294000E8000E94B012ACC08111AAC010918203AD
:102950001F778091E3008078812B8093E300809142
:10296000E800877F8093E8000E94B0128091E80021
:1029700080FFFCCF8091E30080688093E300111119
:1029800002C082E001C083E080937F0389C0805849
:10299000823008F085C080918203909183038C3D42
:1029A00053E0950779F583E08A838AE289834FB7FC
:1029B000F894DE01139620E03EE051E2E32FF0E0D0
:1029C00050935700E49120FF03C0E295EF703F5F02
:1029D000EF708E2F90E0EA3010F0C79601C0C096DD
:1029E0008D939D932F5F243149F74FBF8091E8006D
:1029F000877F8093E8006AE270E0CE0101960E9432
:102A00004F1316C06091840370918503AE014F5F30
:102A10005F4F0E940F12BC01892B09F441C09091B5
:102A2000E800977F9093E80089819A810E94AA1319
:102A30008091E8008B778093E80032C0803881F580
:102A40008091E800877F8093E80080917B038093EA
:102A5000F1008091E8008E7772CF811121C08091C2
:102A600082039091830399270297D4F48091E80020
:102A7000877F8093E8008091820380937B030E948C
:102A8000B01280917B03811106C08091E30087FD25
:102A900002C081E001C084E080937F030E94661041
:102AA0008091E80083FF0AC08091E800877F8093CF
:102AB000E8008091EB0080628093EB00AA960FB64D
:102AC000F894DEBF0FBECDBFDF91CF911F91089567
:102AD0000E94C5150E94C815E0EEF0E0808181607B
:102AE0008083E8EDF0E080818F77808319BCE3E696
:102AF000F0E080818160808310927E0308950E94BF
:102B0000C5150E94C8158091D8008F778093D80092
:102B10008091D80080688093D8008091D8008F7D04
:102B20008093D80084E089BD86E089BD09B400FEA9
:102B3000FDCF10927F0310927B0310927D031092C1
:102B40007C0342E060E080E00E947B128091E10023
:102B50008E7F8093E1008091E20081608093E200AB
:102B60008091E20088608093E2008091E0008E7F97
:102B70008093E0000895E3E6F0E080818E7F80831B
:102B800081E080937E030C947F151092E2000895FB
:102B90001092E10008951F920F920FB60F92112428
:102BA0002F933F934F935F936F937F938F939F9355
:102BB000AF93BF93EF93FF938091E10082FF0BC02F
:102BC0008091E20082FF07C08091E1008B7F8093BB
:102BD000E1000E9475168091E10080FF19C080918C
:102BE000E20080FF15C08091E2008E7F8093E200BA
:102BF0008091E20080618093E2008091D800806241
:102C00008093D80019BC85E080937F030E94361121
:102C10008091E10084FF30C08091E20084FF2CC0ED
:102C200084E089BD86E089BD09B400FEFDCF8091B6
:102C3000D8008F7D8093D8008091E1008F7E8093B3
:102C4000E1008091E2008F7E8093E2008091E200BB
:102C500081608093E20080917B03882311F084E0FF
:102C600007C08091E30087FD02C081E001C083E0DE
:102C700080937F030E944B118091E10083FF24C069
:102C80008091E20083FF20C08091E100877F8093E4
:102C9000E10082E080937F0310927B038091E1004A
:102CA0008E7F8093E1008091E2008E7F8093E2002E
:102CB0008091E20080618093E20042E060E080E089
:102CC0000E947B120E946510FF91EF91BF91AF911E
:102CD0009F918F917F916F915F914F913F912F9134
:102CE0000F900FBE0F901F9018950895CF9380916D
:102CF0007F038823A1F0C091E900CF709091EC0090
:102D0000892F817090FD80E8C82B1092E900809196
:102D1000E80083FD0E940814CF70C093E900CF91B2
:102D200008959093800280937F020895E0917F023E
:102D3000F0918002309721F00190F081E02D09940C
:102D400080E00895EF92FF920F931F93CF93DF934C
:102D5000E0917F02F09180023097B1F18C01028006
:102D6000F381E02D09958091750382FF2DC080FFCE
:102D700004C088E097E00E94A305E80110E282E029
:102D8000E82E87E0F82E8091750380FF0BC08881C4
:102D90001F928F93FF92EF920E943C060F900F902C
:102DA0000F900F90115021961111EDCF8091750366
:102DB00080FF0AC080E097E0DF91CF911F910F91D3
:102DC000FF90EF900C94A305DF91CF911F910F918D
:102DD000FF90EF900895CF93DF9320917D02309183
:102DE0007E022817390709F190937E0280937D02B5
:102DF000E0917F02F09180023097B9F0EC010680FB
:102E0000F781E02D09958091750382FF0EC080FF48
:102E10000CC0DF93CF9382EF96E09F938F930E9435
:102E20003C060F900F900F900F90DF91CF91089577
:102E3000CF93DF9320917B0230917C0228173907D2
:102E400009F190937C0280937B02E0917F02F091E4
:102E500080023097B9F0EC010084F185E02D0995EE
:102E60008091750382FF0EC080FF0CC0DF93CF936B
:102E700082EE96E09F938F930E943C060F900F90F6
:102E80000F900F90DF91CF9108950C94EE170E9450
:102E90008C230C94CD0ABF92CF92DF92EF92FF92D7
:102EA0000F931F93CF93DF9300D000D01F92CDB725
:102EB000DEB70E94F70A02E812E0F12C8F2D0E9483
:102EC000DA0AB82EF801C080C82639F4F3940F5FEF
:102ED0001F4FF0E1FF12F2CF30C08091750381FDEA
:102EE0000E94EF17D12CEE24E3948C2D8E21F9F063
:102EF000D982FA8291E08B2D8E2109F490E09B8398
:102F00000E9495238160782F9D838C8349815A810B
:102F10006B818D810E94251849815A816B817C814A
:102F20008D810E942D23F80180818E258083D3948A
:102F3000EE0CF8E0DF12D9CFC9CF8FEF89838A83F7
:102F40001B820E9495238160782F9D838C83498109
:102F50005A816B818D810E9425180E942C230E942A
:102F6000961690918102891741F10E9496168093DE
:102F700081029091750392FF0EC090FF0CC01F92CA
:102F80008F9383E197E09F938F930E943C060F906D
:102F90000F900F900F90809181020F900F900F90E3
:102FA0000F900F90DF91CF911F910F91FF90EF90B5
:102FB000DF90CF90BF900C943E230F900F900F9016
:102FC0000F900F90DF91CF911F910F91FF90EF9095
:102FD000DF90CF90BF9008950C94E80A0895EF9287
:102FE000FF920F931F93CF93DF938CE297E00E94A1
:102FF000A305C0E0D0E08CE2E82E81E0F82E0EE1DF
:1030000017E08C2F0E94DA0A0E941A23FF92EF9297
:103010001F928F93DF93CF931F930F930E943C06D1
:1030200021968DB79EB708960FB6F8949EBF0FBE37
:103030008DBFC031D10529F7DF91CF911F910F913D
:10304000FF90EF90089508950895CF93DF93CDB743
:10305000DEB72B970FB6F894DEBF0FBECDBF942F0F
:103060004F83252F588769877A878B874A855B85A9
:10307000452B31F02F3F31F481E09F3F19F403C01D
:1030800081E001C080E080FD07C04F8158856985DF
:103090007A858B850E942D23DE01119686E0FD0145
:1030A00011928A95E9F785E0FE01379601900D921D
:1030B0008A95E1F749815A816B817C818D819E815E
:1030C0000E941C1F2B960FB6F894DEBF0FBECDBF1B
:1030D000DF91CF910895CF93882309F465C0C82F5D
:1030E0008CEF8C0F813A20F080E58C0F8E3248F403
:1030F0008C2F0E946625811157C08C2F0E941022B0
:103100000CC080E28C0F883058F4C77081E001C099
:10311000880FCA95EAF70E94B522CF910C94EF224E
:103120008BE58C0F833078F4C53A29F0C63A31F03C
:1031300083E890E005C081E890E002C082E890E07A
:10314000CF910C94EB1688E58C0F873168F5C83A5F
:1031500089F0C93A91F0CA3A99F0CB3AA1F0CC3A49
:10316000A9F0CD3AB1F0CE3AB9F0CF3AC1F080E053
:1031700090E017C082EE90E014C089EE90E011C09C
:103180008AEE90E00EC085EB90E00BC086EB90E0FD
:1031900008C083EB90E005C084EB90E002C087EBB1
:1031A00090E0CF910C941817CF910895882349F19E
:1031B0009CEF980F913A20F090E5980F9E3218F40A
:1031C0000E9460220DC090E2980F983058F48770EA
:1031D00091E001C0990F8A95EAF7892F0E94BB22DE
:1031E0000C94EF229BE5980F933020F480E090E060
:1031F0000C94EB16885A873120F480E090E00C9410
:1032000018170895882321F00E94B5220C94EF220C
:103210000895882321F00E94BB220C94EF22089588
:103220000E94D5220E94A4220E94EF2280E090E01A
:103230000E94EB1680E090E00C9418170E94C522C3
:103240000C941019CF92DF92EF92FF920F931F937D
:10325000CF93DF9300D000D01F92CDB7DEB76C01C3
:103260000E9440238111EAC285E0F601DE01119639
:1032700001900D928A95E1F7F601408151812381F9
:1032800034812115310531F05F3F31F481E04F3F4A
:1032900019F403C081E001C080E080FDCFC2F601D7
:1032A000F280E580E2948FE0E82249835A83FB8232
:1032B000722F3D832C836F2D8D810E9485218C017F
:1032C0000E9484210E947420E12FE295EF708E2FDE
:1032D00090E0FC01E35DFE4F0C94CA25812F807FB6
:1032E0001F70882311F01295107FFF2049F01123E1
:1032F00009F43BC2812F0E94C8220E94EF2235C2EE
:10330000802F0E94D618112309F498C2812F0E94A1
:10331000CE220F900F900F900F900F90DF91CF91D2
:103320001F910F91FF90EF90DF90CF900C94EF22C0
:10333000812F807F1F70803211F01295107F002343
:1033400019F0013009F12BC0FF20A9F0EE2059F14E
:10335000F1E0812FEF1228C00F900F900F900F9087
:103360000F90DF91CF911F910F91FF90EF90DF9021
:10337000CF900C94D822EE2021F021E0E21609F43F
:103380005DC20E94DB222DC0FF20E9F085E08E1592
:1033900008F454C20E94B222812329F022C0FF20E7
:1033A000F1F0E11015C0812F0F900F900F900F904A
:1033B0000F90DF91CF911F910F91FF90EF90DF90D1
:1033C000CF900C94021994E09E1508F437C209C0FE
:1033D000F601858180FFC9C18F708583E4CFE1103C
:1033E000D7C1812F4AC1812F86958695837019F0A8
:1033F0008130B9F023C2FF2019F0C801937002C0D8
:1034000080E090E00F900F900F900F900F90DF9161
:10341000CF911F910F91FF90EF90DF90CF900C9480
:10342000EB16FF2019F0C801937002C080E090E015
:103430000F900F900F900F900F90DF91CF911F91F1
:103440000F91FF90EF90DF90CF900C941817812F81
:10345000837009F070C0F110F1C1202F22952695DC
:103460002770220F220F602F6F70862F90E0A0E050
:10347000B0E06C017D01022E04C0CC0CDD1CEE1C02
:10348000FF1C0A94D2F704FF12C08FE090E0A0E086
:10349000B0E004C0880F991FAA1FBB1F2A95D2F75E
:1034A000BC01CD01609570958095909503C060E05A
:1034B00070E0CB011695169513701230B1F040F5FF
:1034C0006C297D298E299F29113031F10F900F90A1
:1034D0000F900F900F90DF91CF911F910F91FF9060
:1034E000EF90DF90CF900C9499206C297D298E2944
:1034F0009F290F900F900F900F900F90DF91CF9119
:103500001F910F91FF90EF90DF90CF900C94B3201C
:103510000E949920C701B6010F900F900F900F9055
:103520000F90DF91CF911F910F91FF90EF90DF905F
:10353000CF900C947F20FF2019F0812F817001C063
:103540008695882309F47AC1202F22952695277025
:10355000220F220F602F6F70862F90E0A0E0B0E066
:103560006C017D01022E04C0CC0CDD1CEE1CFF1C86
:103570000A94D2F704FF12C08FE090E0A0E0B0E020
:1035800004C0880F991FAA1FBB1F2A95D2F7BC0140
:10359000CD01609570958095909503C060E070E0D6
:1035A000CB011695169513701230B1F040F56C29C9
:1035B0007D298E299F29113031F10F900F900F90A6
:1035C0000F900F90DF91CF911F910F91FF90EF908F
:1035D000DF90CF900C9460216C297D298E299F2942
:1035E0000F900F900F900F900F90DF91CF911F9140
:1035F0000F91FF90EF90DF90CF900C9472210E947A
:103600006021C701B6010F900F900F900F900F909F
:10361000DF91CF911F910F91FF90EF90DF90CF90AE
:103620000C944E21003FC1F128F480E4800F8032D9
:1036300050F096C0023F09F45EC008F449C0033F51
:1036400009F46CC08DC0F02FF071EF2E812F8F71B7
:10365000FF2051F00E94E720802FEE2019F0829584
:10366000807FA2CE8F70A0CE0E940821802FEE20F6
:1036700019F08295807F01C08F700F900F900F908E
:103680000F900F90DF91CF911F910F91FF90EF90CE
:10369000DF90CF900C940919FF20A9F024E02E159B
:1036A00008F4CCC0812F8F710F900F900F900F9066
:1036B0000F90DF91CF911F910F91FF90EF90DF90CE
:1036C000CF900C942D2185E08E1508F4B7C0EACF79
:1036D000FF2099F0812F8F710F900F900F900F9016
:1036E0000F90DF91CF911F910F91FF90EF90DF909E
:1036F000CF900C94E720FF2069F3812F8F710F90FA
:103700000F900F900F900F90DF91CF911F910F911D
:10371000FF90EF90DF90CF900C940821FF2089F06C
:10372000812F8F710F900F900F900F900F90DF915E
:10373000CF911F910F91FF90EF90DF90CF900C945D
:10374000D2200F900F900F900F900F90DF91CF919C
:103750001F910F91FF90EF90DF90CF900C94CD20B0
:10376000FF2099F0EE2009F4B5CF802F0F900F9035
:103770000F900F900F90DF91CF911F910F91FF90BD
:10378000EF90DF90CF900C946B18EE2009F4B5CF3A
:10379000802F0F900F900F900F900F90DF91CF918F
:1037A0001F910F91FF90EF90DF90CF900C94D6185F
:1037B000412F4F70602FC6010E9401240F900F907F
:1037C0000F900F900F90DF91CF911F910F91FF906D
:1037D000EF90DF90CF900C94CF1F01112FC0FF20EE
:1037E00069F10E941E199FEFE0E7F2E09150E0407E
:1037F000F040E1F700C000000F900F900F900F9085
:103800000F90DF91CF911F910F91FF90EF90DF907C
:10381000CF900C94E223412F4F70602FC6010F9080
:103820000F900F900F900F90DF91CF911F910F91FC
:10383000FF90EF90DF90CF900C9404240F900F90A6
:103840000F900F900F90DF91CF911F910F91FF90EC
:10385000EF90DF90CF9008951F93CF93DF9300D028
:1038600000D01F92CDB7DEB7942F4983252F5A83FE
:103870006B837C838D834C815D81452B31F02F3FA1
:1038800031F481E09F3F19F403C081E001C080E082
:10389000182F117080FD31C049815A816B817C8164
:1038A0008D810E948521292F22952F702C3030F494
:1038B0002A30A0F42250223030F022C02C30C9F03F
:1038C0002F30B9F01DC0853A28F48430C0F482301E
:1038D00028F415C090E2980F983088F0883E30F4B4
:1038E000803E68F48450813A58F409C0803F41F426
:1038F00006C093FB112710F903C010E001C011E0CE
:10390000812F0F900F900F900F900F90DF91CF911C
:103910001F910895CF93DF9300D000D01F92CDB7B1
:10392000DEB70F900F900F900F900F90DF91CF9117
:103930000895CF93DF9300D000D000D0CDB7DEB78D
:1039400026960FB6F894DEBF0FBECDBFDF91CF91A4
:103950000895CF93DF93C091920280919302C8178C
:10396000A1F0D0E0CE0166E070E00E94B925FC0134
:10397000EC56FD4F40815181628173818481958134
:103980000E94991C2196C770E8CFDF91CF910895CE
:103990004091C4025091C5026091C6027091C70265
:1039A0008091C8029091C9020C94991C1F93CF93E7
:1039B000DF938091C90282958F7009F05CC080917D
:1039C000C602882309F457C02091920210919302F5
:1039D000C091C402D091C502A091C702B091C802A3
:1039E00081E0CF3F09F080E0482F211709F443C060
:1039F000109721F0DF3F21F080E003C081E001C09B
:103A0000842F30E080FD33C0C90166E070E00E9481
:103A1000B925FC01EC56FD4F81818D1328C08081B2
:103A20008C1325C08281811122C0838194818A1BDD
:103A30009B0B883C9105D8F48091C9028F708061FE
:103A40008093C902C90166E070E00E94B925FC01BB
:103A5000E756FD4F90819F709061908384EC92E0D7
:103A60000E942219DF91CF911F910C94A91C2F5F06
:103A70003F4F2770BACFDF91CF911F9108959F924A
:103A8000AF92BF92CF92DF92EF92FF920F931F936C
:103A9000CF93DF93CDB7DEB761970FB6F894DEBF53
:103AA0000FBECDBF8C0185E0F801DE011D960190AF
:103AB0000D928A95E1F7F80140812181F280C3805F
:103AC000D4809091C4023091C5026091C702709178
:103AD000C8026115710531F03F3F31F481E09F3F2D
:103AE00019F403C081E001C080E0F82FF1709F2E2F
:103AF00080FD59C184ECA82E82E0B82EE090C60269
:103B0000F601E61BF70BEE2009F4EDC08091C90227
:103B1000582F507FE83CF10508F0A7C0511156C05E
:103B2000231313C0491311C0EF2CF1100EC08F7076
:103B300080618093C9020E94C81CC5010E9422199D
:103B40008091C902F801858364C1C114D10431F0A8
:103B50002F3F31F481E04F3F19F403C081E001C0F1
:103B600080E080FD03C081E08F2502C080E090E00E
:103B7000F82FF170EF2E80FF1FC0E091920230917C
:103B80009302E31709F421C1F0E0CF0166E070E091
:103B90000E94B925DC01AC56BD4F11968C9111974E
:103BA000281307C08C91481304C012968C91F81208
:103BB00003C03196E770E5CFEF2CFF2009F429C14F
:103BC0008091C90281608093C90264C0231306C03A
:103BD000491304C0F11002C0F801A9C04D872E8717
:103BE000FF867C2DD98AC88A522F6F2D89890E9421
:103BF0002C1C8823A1F1FF2091F12091C902822F72
:103C000082958F7090E0029774F08091C402909139
:103C1000C50298878F831986DB86CA862C87CE01DA
:103C200007960E94221986E0F801A4ECB2E0019008
:103C30000D928A95E1F70E94D61C0E94C81C12C002
:103C4000231751F14D872E87FF867C2DD98AC88A8C
:103C5000522F6F2D89890E942C1C81112CC0C80104
:103C60000E942219EE24E394D4C05111E9CF7C2D97
:103C7000D98AC88A522F6F2D89890E948A1C84ECA8
:103C800092E00E94221986E0F50111928A95E9F7E7
:103C90000E94C81CE12CBDC04913D4CFF110D2CF73
:103CA000F8018583C8010E94221986E0F50111926E
:103CB0008A95E9F7AEC0FF2091F22091C902822FC8
:103CC00082958F7090E002970CF4ADCF8091C40282
:103CD0009091C5029A8389831B82DD82CC822E83D8
:103CE000CE0101969ECFE83CF10508F04CC0EF2CC8
:103CF000FF2009F4B4CF231330C049132EC0209104
:103D0000C90220FD21C0822F82958F70482F50E07C
:103D100041155105C9F0F80125834F30510541F097
:103D20008F5F982F9295907F822F8F70892B85833C
:103D3000C8010E94221986E0F801A4ECB2E00190CB
:103D40000D928A95E1F72CC086E0F801A4ECB2E070
:103D500001900D928A95E1F75CC04D872E87FF8612
:103D60007C2DD98AC88A522F6F2D89890E942C1CDC
:103D7000811159CF8091C90281608093C902C80125
:103D80000E94221946C07C2DD98AC88A522F6F2DD5
:103D900089890E948A1C86E0F50111928A95E9F7CB
:103DA0000E94C81C36C0FF2009F459CF4D872E87CA
:103DB000FF867C2DD98AC88A522F6F2D89890E944F
:103DC0002C1C882309F44BCF2ECF7C2DD98AC88A8E
:103DD000522F6F2D89890E948521292F22952F70BE
:103DE000223028F49F7039F0811105C00BC02430B7
:103DF00028F49F7049F4805E883020F0C8010E944A
:103E000022199E2CE92C05C0F8019581907F99F725
:103E1000F9CF8E2D61960FB6F894DEBF0FBECDBFE1
:103E2000DF91CF911F910F91FF90EF90DF90CF9096
:103E3000BF90AF909F900895CF93DF93CDB7DEB73B
:103E40002C970FB6F894DEBF0FBECDBF4F835887B7
:103E500069877A878B879C87CE0107960E943F1DD2
:103E60008823D1F09F8188852A853B85232B31F0DB
:103E70008F3F31F481E09F3F19F403C081E001C01E
:103E800080E080FD6FC04F81588569857A858B857C
:103E90009C850E94991C66C086E0FE013796DE0173
:103EA000119601900D928A95E1F7FF81E8856A8568
:103EB0007B856115710531F0EF3F31F481E0FF3F03
:103EC00019F403C081E001C080E080FD4BC0809107
:103ED000930290E09C012F5F3F4F27703327409162
:103EE000920250E02417350709F443C0F983EA83AE
:103EF0007D836C8366E070E00E94B925DC01AC56DE
:103F0000BD4F96E0FE01319601900D929A95E1F732
:103F1000209393020E94A91C25C090E066E070E007
:103F20000E94B9258C569D4F0E943F1D882371F138
:103F30008091920290E066E070E00E94B925FC0159
:103F4000EC56FD4F4081518162817381848195815E
:103F50000E94991C8091920290E0019687709927A7
:103F60008093920280919202909193028913D5CF0F
:103F70000DC00E941E191092930210929202E4EC5E
:103F8000F2E086E0DF011D928A95E9F72C960FB6E4
:103F9000F894DEBF0FBECDBFDF91CF910895DF92C1
:103FA000EF92FF920F931F93CF93DF93FC01892B26
:103FB00009F488C0E12CF12CDD24D394EF01219683
:103FC0008491853709F460C058F4843708F04EC0F6
:103FD000843008F068C08130D1F0823071F172C055
:103FE000883709F45BC050F4863709F453C087372B
:103FF00009F068C08E2D0E94C22252C09CE7980F23
:10400000903708F05FC08F770E94D6184EC08F019E
:104010000E5F1F4FFE01849190E2980F983050F48C
:104020008770FD2D01C0FF0F8A95EAF78F2F0E9440
:10403000C82215C00E946B1814C08F010E5F1F4F5D
:10404000FE01849190E2980F983068F48770FD2DFE
:1040500001C0FF0F8A95EAF78F2F0E94CE220E949F
:10406000EF22E80122C00E94D618FBCFCF010296B2
:10407000FE01C491CC2361F0EFE9FFE03197F1F745
:1040800000C00000C150F6CFCF010296FE01F490AF
:10409000EC010BC00E94B222E82E07C00E94C5228C
:1040A0000E94EF2202C00E946B188F2D882341F0DE
:1040B000EFE9FFE03197F1F700C000008150F6CF43
:1040C000FE017CCFDF91CF911F910F91FF90EF9078
:1040D000DF90089560934A0370934B0380934C03E1
:1040E00090934D030C943D23089560934E03709379
:1040F0004F0380935003909351030C943C230F93F0
:104100001F9300914E0310914F0320915003309163
:104110005103602B712B822B932B60934E03709372
:104120004F0380935003909351031F910F910C9470
:104130003C230F931F9300914E0310914F03209146
:1041400050033091510360237123822393236093A2
:104150004E0370934F0380935003909351031F912C
:104160000F910C943C230F931F9300914E031091D9
:104170004F0320915003309151036027712782270C
:10418000932760934E0370934F0380935003909353
:1041900051031F910F910C943C2360E070E0CB0120
:1041A0000C946A200F931F9341E050E060E070E0B0
:1041B0008A019B0104C0000F111F221F331F8A9523
:1041C000D2F7C901B8011F910F910C946A200F9387
:1041D0001F9341E050E060E070E004C0440F551FC1
:1041E000661F771F8A95D2F780914A0390914B03FF
:1041F000A0914C03B0914D038A019B01082B192B10
:104200002A2B3B2BC901B8011F910F910C946A20F6
:104210000F931F9341E050E060E070E004C0440F52
:10422000551F661F771F8A95D2F740955095609568
:10423000709580914A0390914B03A0914C03B091EB
:104240004D038A019B01082319232A233B23C9011B
:10425000B8011F910F910C946A200F931F9341E0B6
:1042600050E060E070E004C0440F551F661F771FE8
:104270008A95D2F780914A0390914B03A0914C0309
:10428000B0914D038A019B01082719272A273B2754
:10429000C901B8011F910F910C946A200F931F93CD
:1042A00000914A0310914B0320914C0330914D0330
:1042B000602B712B822B932B1F910F910C946A20F2
:1042C0000F931F9300914A0310914B0320914C03CD
:1042D00030914D0360237123822393231F910F910B
:1042E0000C946A200F931F9300914A0310914B0383
:1042F00020914C0330914D0360277127822793272B
:104300001F910F910C946A2008958F929F92AF9203
:10431000BF92DF92EF92FF920F931F93CF93DF93A1
:1043200000D000D01F92CDB7DEB76B837C838D8326
:104330008A018C819D81892B31F01F3F31F481E00E
:104340004F3F19F403C081E001C080E080FF03C04B
:1043500080E090E054C08B81882309F43DC08090B8
:104360004A0390904B03A0904C03B0904D03809172
:104370004E0390914F03A0915003B0915103882AAE
:10438000992AAA2ABB2A2FE1E22EF12CD501C401D9
:104390000E2C04C0B695A795979587950A94D2F7E9
:1043A00080FD06C081E0E81AF10880F7D12C07C033
:1043B000DE2CB8018E2D0E944506019799F3E12F5E
:1043C000F0E093E0EE0FFF1F9A95E1F7E653FD4F03
:1043D000E00FF11DD0820CC0E12FF0E083E0EE0F82
:1043E000FF1F8A95E1F7E653FD4FE00FF11DD080E6
:1043F00009831A8369817A818D2D0E9445060F9069
:104400000F900F900F900F90DF91CF911F910F9110
:10441000FF90EF90DF90BF90AF909F908F900895A6
:1044200090911401992379F190911501992359F1F3
:10443000982F9695969596959F31A1F0E09116014B
:10444000F0911701E90FF11D877021E030E0A9011B
:1044500002C0440F551F8A95E2F7CA019181892B4A
:10446000818308959091750390FF29C01F928F93C7
:1044700088E597E09F938F930E943C060F900F90E2
:104480000F900F9008952091160130911701F901B6
:1044900032969FEF40E05191851789F09F3F19F4C4
:1044A000511101C0942F4F5F4E31A9F79F3F39F052
:1044B000F901E90FF11D97FDFA958283089508959A
:1044C00090911401992381F190911501992361F143
:1044D000982F9695969596959F31A9F0E0911601A3
:1044E000F0911701E90FF11D877021E030E0A9017B
:1044F00002C0440F551F8A95E2F7CA018095918149
:104500008923818308959091750390FF1CC01F92A9
:104510008F938AE397E09F938F930E943C060F90BE
:104520000F900F900F900895E0911601F0911701F0
:104530009F01225E3F4F9281891301C01282319602
:10454000E217F307C1F7089581E090E0E0911601CA
:10455000F0911701E80FF91F108201968032910542
:10456000A9F7089580917403089590917403892B9D
:1045700080937403089580959091740389238093A8
:10458000740308958093740308951092740308953A
:1045900090917303892B8093730308958095909174
:1045A000730389238093730308951092730308950E
:1045B000809352030895109252030895809116013A
:1045C00090911701FC0131969C01205E3F4F80E0E5
:1045D000919191118F5FE217F307D1F70895E09160
:1045E0001601F0911701809174038083E091160108
:1045F000F0911701908180917303892B80838091C2
:104600005203882361F0E0911601F0911701908127
:10461000892B80830E94DE228111109252038091A7
:104620001601909117010C94A21690933501809376
:10463000340108958295982F9373292F220F220F0A
:10464000982F9C7C96959695922B892F8575880F2F
:104650009A7A9695892B08950895CF93DF9300D089
:1046600000D01F92CDB7DEB70F900F900F900F9034
:104670000F90DF91CF910895089508950C94EC1751
:1046800080E0089583B7817F8C6083BF83B78160AA
:1046900083BF7894889583B78E7F83BF0895CF9327
:1046A0000E9423180E94F70A0E942418C0E08C2F51
:1046B0000E94DA0A811104C0CF5FC031C1F701C086
:1046C00081E0CF9108950E94E00A0C941E191F9278
:1046D0000F920FB60F9211248F939F93AF93BF93B6
:1046E0008091760390917703A0917803B09179033C
:1046F0004196A11DB11D8093760390937703A093FB
:104700007803B0937903BF91AF919F918F910F90F0
:104710000FBE0F901F90189582E084BD93E095BD69
:104720009AEF97BD80936E0008952FB7F89480910B
:10473000760390917703A0917803B09179032FBF0E
:1047400008952FB7F8946091760370917703809164
:104750007803909179032FBF08959C014FB7F89487
:104760008091760390917703A0917803B0917903BB
:104770004FBF821B930B089578941F920F920FB630
:104780000F9211248F939F93AF93BF9380917603E1
:1047900090917703A0917803B09179030196A11DC0
:1047A000B11D8093760390937703A0937803B09321
:1047B0007903BF91AF919F918F910F900FBE0F9092
:1047C0001F9018950E946815F89487E797E79093D3
:1047D00001088093000887E090EBDC018093880358
:1047E00090938903A0938A03B0938B039CE088E1A4
:1047F0000FB6F894A895809360000FBE9093600068
:10480000FFCF80E090E008950895CF93C82F1F92C6
:104810008F938CE797E09F938F930E943C0681E0F3
:1048200090E0A0E0B0E0BC01CD0104C0660F771FAE
:10483000881F991FCA95D2F70E9475200F900F907C
:104840000F900F90CF910C941E19CF938732A8F53B
:104850008E3108F02BC1803109F49FC0F8F4873005
:1048600009F464C0A8F4863009F024C1809175036E
:10487000817F8E7F8093750381E897E00E94A30576
:1048800084E69AE00E94A30581E080937A034CC0FD
:104890008B30F1F18E3009F46CC00CC1863109F413
:1048A000B0C020F4813109F4EDC004C1893109F4AC
:1048B00091C08B3109F449C0FDC0883349F150F4EF
:1048C000893209F4F1C0853309F4EEC0873209F06A
:1048D000F1C0EAC0833409F4E7C028F48A3308F44D
:1048E000E9C08953E4C0883409F0E4C00E941E196D
:1048F00083E59AE00E94A3052FEF83ED90E321501A
:1049000080409040E1F700C000000E94E2230CC00C
:104910008CE997E05CC08AE39AE00E94A30580914D
:104920007503816080937503C1E0C9C080917503F0
:10493000C82FC17080FFEFCF86E49AE00E94A305E4
:1049400080917503817F8E7F3DC09091750391FBAF
:10495000CC27C0F981E0C827892FC0FB81F980935B
:104960007503CC2319F08DE29AE027C08FE19AE01D
:104970002EC09091750392FBCC27C0F981E0C82727
:10498000892FC0FB82F980937503CC2319F080E155
:104990009AE013C080E09AE01AC09091750393FBEF
:1049A000CC27C0F981E0C827892FC0FB83F9809309
:1049B0007503CC2351F084EF99E00E94A305809108
:1049C00075038160809375037AC087EE99E00E9439
:1049D000A305AACF88ED99E00E94A30582EB99E098
:1049E0000E94A3058AE699E00E94A30582E499E06B
:1049F0000E94A30586EF98E00E94A3058AEC98E048
:104A0000E6CF8CEB98E00E94A3050E9496161F92B9
:104A10008F9382EA98E09F938F930E943C06809147
:104A200014011F928F938BE898E09F938F930E94BD
:104A30003C0680917A021F928F9388E798E09F93BB
:104A40008F930E943C06809115011F928F9385E6FB
:104A500098E09F938F930E943C060E94A1239F930E
:104A60008F937F936F938EE498E09F938F930E9430
:104A70003C068DB79EB746960FB6F8949EBF0FBE04
:104A80008DBF52CF0E941E19C091150181E0C82729
:104A9000C0931501CC2329F084E498E00E94A3057B
:104AA0000EC089E398E093CF80E001C08D510E9451
:104AB00005243ACF87E398E00E94A305C0E08C2F3D
:104AC000CF91089580E008950C946225CF93C82F6C
:104AD00080917A03882319F0813059F042C0E09127
:104AE0001601F09117018081823261F08434D9F58A
:104AF00009C0E0911601F09117018081823211F016
:104B0000843461F48C2F0E946425811104C08C2FA1
:104B10000E94252424C081E090E021C08C2F0E94B7
:104B2000622581111BC0C43189F018F4CB3029F003
:104B300010C0C93259F0C83361F481E897E00E948F
:104B4000A30588E797E00E94A30508C010927A03A6
:104B50000CC086E797E00E94A30507C081E0817042
:104B600006C010927A0380E002C080E0F8CFCF91B7
:104B700008950024552704C0080E591F880F991F57
:104B8000009729F076956795B8F37105B9F7802DF0
:104B9000952F0895EE0FFF1F0590F491E02D0994D5
:044BA000F894FFCFB7
:104BA4000080FFFF0559010000FFA20E0F0FA50EA4
:104BB400DA0EA60E0101530340362239A2066C0612
:104BC4004A0611069D05B605CF05EF05000008004D
:044BD40004000200D7
:106800008800EA44E944E244040005000600070069
:10681000080009000A000B000C000D000E000F001C
:1068200010001100120013001400150016001700CC
:10683000180019001A001B001C001D001E001F007C
:10684000200021002200230024002500260027002C
:10685000280029002A002B002C002D002E002F00DC
:10686000300031003200330034003500360037008C
:10687000380039003A003B003C003D003E003F003C
:1068800040004100420043004400450046004700EC
:10689000480049004A004B004C004D004E004F009C
:1068A000500051005200530054005500560057004C
:1068B000580059005A005B005C005D005E005F00FC
:1068C0006000610062006300640065A185006700EC
:1068D000680069006A006B006C006D006E006F005C
:1068E0007000710072007300890087008A008B00BD
:1068F000E000E100E200E300E400E500E600E7007C
:106900000100010001000100EA4401000100E2442D
:106910000100010001000100460001004A004B0097
:10692000010001004700480001000100E9440100A6
:106930000100010001000100010001003A003B00DC
:106940003C003D003E003F0040004100420043004B
:10695000010035004C0039000100440045005200A0
:1069600049000100010050004F0029004D004E0079
:1069700051000100010001000100010001000100BF
:1069800001000100010001000100010001000100FF
:1069900001000100010001000100010001004D00A3
:1069A0004A004E004B0001000100010001000100FF
:1069B00001000100010001000100010001000100CF
:1069C00001000100010001000100010001000100BF
:1069D00001000100010001000100010001000100AF
:1069E0000100010001000100490001000100010057
:1069F000010001000100010001000100010001008F
:00000001FF
